:020000040800F2
:100000003006002085090008A1090008A50900089C
:10001000A9090008AD090008B109000800000000A6
:10002000000000000000000000000000B50900080A
:10003000B909000800000000BD090008C109000856
:10004000C5090008C9090008CD090008D109000840
:10005000D5090008D9090008DD090008E1090008F0
:10006000E5090008E9090008ED090008F1090008A0
:10007000F5090008F9090008FD090008010A00084F
:10008000050A0008090A00080D0A0008110A0008FC
:10009000150A0008190A00081D0A0008210A0008AC
:1000A000250A0008290A00082D0A0008310A00085C
:1000B000350A0008390A00083D0A0008410A00080C
:1000C000450A0008490A00084D0A0008510A0008BC
:1000D000550A0008590A00085D0A0008610A00086C
:1000E000650A0008690A00086D0A0008710A00081C
:1000F000750A0008790A00087D0A0008810A0008CC
:10010000850A0008890A00088D0A0008910A00087B
:10011000950A0008990A00089D0A0008A10A00082B
:10012000A50A0008A90A0008AD0A0008B10A0008DB
:1001300010B5DFF8DC4325220021204600F018FA34
:1001400004F11000DFF8CC1301600022827410BDAE
:10015000DFF8BC0390F8220000B1012070470000D6
:1001600070B5FFF7E5FFDFF8A843DFF8AC53DFF821
:10017000AC63DFF8AC230FF271110FF2AD006560D4
:10018000266000F00FF994F8220050B960682168E9
:10019000814206D2A94204D3B04202D800BF012056
:1001A00070BD002070BD80B5FFF7C2FF00220021A6
:1001B0000FF2491000F0F6F8D54890F82210481ECA
:1001C0008041C00F02BD38B5FFF7B2FF00F0F8F96B
:1001D000D14CCF4D204600F01AFA85F8220004F5E4
:1001E000006460B9CF488442F4D30FF26910002252
:1001F000002100F0D7F8BDE8314000F0EFB931BD83
:1002000080B500F0E2FAC448C74A416800910099FD
:10021000136843F0007313605060006880F308882F
:10022000BDE801400847000070B5B94C6169A08B7A
:1002300094F8205041186068814228BF08466060E9
:100240002068814288BF01462160A90805EB5172F0
:10025000D208B5EBC2001AD1B4F91E1000293FDD57
:1002600000F09EF800F023F9A06994F8241000EB48
:10027000102202EB104202EB1060401884F82400B8
:100280000022E08BA261A0F10801E183E4E721698B
:100290000020083984F8240021612D1D00261DE06E
:1002A0002169022204F1080000F086F9207A3A2838
:1002B00004D0022104F1080000F0EAF8207A617A03
:1002C00000012072761C081820722069217A801C97
:1002D000206194F82400081884F82400AE42DFD38B
:1002E000BDE87040FAE0000090480168027C0B0E07
:1002F00003EB114189180174F0E0000070B5844CE3
:100300006669A08B0425861906E0E18BA1F108003F
:100310000021E083361DA161B4F91E10012917DB0D
:1003200000F03EF800F0C3F8B4F91E00A84203DA6A
:1003300000EBD075ED032D0C2A46314604F1180070
:1003400000F0FAF80028E0D0072084F8220070BD01
:1003500022E0000070B56E4C6569A08B744E4519A3
:1003600016E000F01DF800F0A2F8A169284600F0A0
:100370008CF984F822000020295C3154401C0928A3
:10038000FADBE08BA0F108010020E1832D1DA061C4
:10039000B4F91E000028E4DCBDE87040022061E0F2
:1003A00008205FE02DE9F843594C80460F469146FE
:1003B000012604F1210521695E4A914230D20120D3
:1003C00000F050F8207A3A2849D1FFF7E9FF607A27
:1003D000217A227BE37A00EB011084F8200094F864
:1003E00020004100E183617B01EB0211A27A01EB65
:1003F000032101EB0231A183A27BE17B01EB02111E
:100400002970A28B2978101800EB12200818E870C8
:1004100021B101291CD0042908D01AE0C04718E0F6
:100420000320687005216970BDE8F183042000F0A5
:1004300019F8617A207AE27A090641EA0071A07A15
:1004400041EA005141EA0241616117B1B84700E059
:100450000026B9F1000F02D0C8470028E4D13000CF
:10046000A9D1E1E770B52A4D29690446224605F174
:10047000080000F0A1F82869297A26183A292E6187
:1004800005D0214605F10800BDE8704000E070BDD0
:1004900010B5002208E0835CA3F130040A2C2CBFC5
:1004A000373B303B8354521C8A42F4DB10BD30B5DD
:1004B000002017490A180B18127A0C1812011A7228
:1004C000657A2A430D1884002A72D2B28B69A24041
:1004D000801C1A4308288A61ECDB30BD38B50C4D0E
:1004E00005F122040220A178C943491CA170FFF73D
:1004F000B9FF687A297A00EB01106070A178607802
:1005000088421CBF062020700021A17031BD000070
:100510000000002000080208002000080000020877
:10052000510100080100020804ED00E01400002061
:10053000280000200108070810B503461046421E97
:1005400038B113F8010B11F8014BA04203D1002878
:10055000F4D1002010BD001B10BD03E011F8013BD9
:1005600000F8013B13465A1E9BB2002BF6D1704790
:10057000130003D00A46194600F032B9704730B470
:10058000002513E050F8042BD30744BFA9F1010361
:100590009A18091F042942F8045BFAD213468C0703
:1005A00044BF15809B1CC90748BF1D7050F8041B31
:1005B0000029E7D130BC704792B2FFF7CEBF0000F0
:1005C00000BF03480349044A01600260704700000D
:1005D0000420024023016745AB89EFCD30B5DFF839
:1005E0007411DFF87401CB68DFF870211C06DFF8A6
:1005F000703144BF0A6008601D8840F20124A542A2
:1006000004D3CB6C1C0644BF0A64086430BD38B503
:100610000446DFF84C01DFF84C51018840F201221A
:1006200091421DD3DFF840319C424FF4702019D322
:1006300000F0ABF8010024D1286C40F002002864DF
:100640006C64E868810748BF6C60286C40F040002B
:10065000286400F017F8296C21F00201296432BDEA
:100660004FF4702000F086F801000AD1286840F0AD
:10067000020028606C6000F043F8296821F0020154
:10068000296032BD4FF470207FE070B500F029F88A
:1006900040F201239A4205460CD300F01DF80BD31B
:1006A00000F073F8010016D1306C40F001003064A6
:1006B0002C601BE04FF4702000F05CF801000AD1C0
:1006C000306840F0010030602C6000F016F83168AE
:1006D00049084900316070BD234988424FF47020B9
:1006E00070470C461E491F4E0A887047FFF7CAFF25
:1006F000316C49084900316470BD4FF4702039E015
:100700004FF47020296841F04001296032E0174918
:100710000A680020D30701D5012070470A68D30674
:1007200001D50320704709684A0748BF0220704777
:100730000F490A680020D30701D5012070470A68D5
:10074000D30601D50320704709684A0748BF022035
:100750007047000004200240AB89EFCD23016745BC
:10076000E0F7FF1F10200240FFFF07080C200240A7
:100770004C20024010B50446FFF7C9FF641E012853
:1007800002D1002CF8D1042010BD10B50446FFF7AB
:10079000CFFF641E012802D1002CF8D1042010BD27
:1007A00080B54FF4C06000F025F80B494CF6CC4002
:1007B000086045F255520A6006234B60C86800285D
:1007C000FCD140F6FF728A6001BD0448002101603F
:1007D00041608160704700000030004010E000E0A0
:1007E0004018491C1CBFB1F1010100F8012DF9D1DD
:1007F00070470000FFE7DFF8181001EB90110123AC
:100800000A6800F01F0003FA00F010430860704708
:100810000010024010B52B49086840F00100086044
:100820004A68294802404A600B68284A13400B6016
:10083000086820F4802008604B68254803404B601E
:100840000C6822400A604FF41F028A60086840F476
:10085000803008604FF6FF700A68401E920301D492
:100860000028F9D10868820300D4FEE74868486090
:100870004A684A60486840F480604860486820F4EC
:1008800040304860486840F4403048604A68114849
:1008900002404A6010484A6802434A600B6843F0CD
:1008A00080730B6008688201FCD54868800880006E
:1008B0004860486840F00200486048680207FCD57C
:1008C00010BD0000001002400C00FFE8FFFFF6FE24
:1008D000FFFF00F7FFFFC3F70000280810B5074926
:1008E00079441831064C7C44163404E00A68081D2B
:1008F000114488470146A142F8D110BD30000000E4
:100900003C00000080B5FFF74BFFFFF729FC0028F3
:1009100007D000BFFFF747FC002802D100BFFFF758
:1009200052FCFFF76DFC002002BD000053FCFFFFEE
:1009300030000000000000200000000000F00DF872
:10094000002801D0FFF7CAFFAFF300800020AFF30B
:100950000080FFF7D7FF00F002F80120704700F099
:1009600001B800000746384600F002F8FBE7000037
:1009700080B5AFF30080024A11001820ABBEFBE740
:10098000260002000148804701480047150800087A
:1009900095090008AFF30080AFF30080FFF7CEFFAA
:1009A000FFF7FEBFFFF7FEBFFFF7FEBFFFF7FEBF7B
:1009B000FFF7FEBFFFF7FEBFFFF7FEBFFFF7FEBF6B
:1009C000FFF7FEBFFFF7FEBFFFF7FEBFFFF7FEBF5B
:1009D000FFF7FEBFFFF7FEBFFFF7FEBFFFF7FEBF4B
:1009E000FFF7FEBFFFF7FEBFFFF7FEBFFFF7FEBF3B
:1009F000FFF7FEBFFFF7FEBFFFF7FEBFFFF7FEBF2B
:100A0000FFF7FEBFFFF7FEBFFFF7FEBFFFF7FEBF1A
:100A1000FFF7FEBFFFF7FEBFFFF7FEBFFFF7FEBF0A
:100A2000FFF7FEBFFFF7FEBFFFF7FEBFFFF7FEBFFA
:100A3000FFF7FEBFFFF7FEBFFFF7FEBFFFF7FEBFEA
:100A4000FFF7FEBFFFF7FEBFFFF7FEBFFFF7FEBFDA
:100A5000FFF7FEBFFFF7FEBFFFF7FEBFFFF7FEBFCA
:100A6000FFF7FEBFFFF7FEBFFFF7FEBFFFF7FEBFBA
:100A7000FFF7FEBFFFF7FEBFFFF7FEBFFFF7FEBFAA
:100A8000FFF7FEBFFFF7FEBFFFF7FEBFFFF7FEBF9A
:100A9000FFF7FEBFFFF7FEBFFFF7FEBFFFF7FEBF8A
:100AA000FFF7FEBFFFF7FEBFFFF7FEBFFFF7FEBF7A
:040AB000FFF7FEBF8F
:040000050800099551
:00000001FF
